:020000040000FA
:04000000C5EF0AF04E
:06002A00D9CFE5FFE1CF94
:10003000D9FF00C0E5FF01C0E5FF02C0E5FF03C036
:10004000E5FF04C0E5FF05C0E5FF06C0E5FF07C00A
:10005000E5FF08C0E5FF09C0E5FF0AC0E5FF020EA5
:10006000DBCF00F0030EDBCF01F0040EDBCF02F09C
:10007000050EDBCF03F0060EDBCF04F0070EDBCF5F
:1000800005F000C006F001C007F002C008F0035000
:1000900003E003500508036E270EE56E100EE56EB3
:1000A0000550E56E0450E56EAAEC05F0096EF3CF3D
:1000B0000AF0040EE126300E092609C0E5FF06C04D
:1000C000E9FF07C0F3FF0850D1EC0AF0062AD8B0C8
:1000D000072AD8B0082A030603500EE12E0EE56E5B
:1000E00006C0E9FF07C0F3FF0850D1EC0AF0062A6A
:1000F000D8B0072AD8B0082A270EE56E100EE56E94
:100100000550E56E0450E56E4EEC05F0046EF3CF3D
:1001100005F0040EE126030EE56EE80EE56E0550CF
:10012000E56E0450E56EAAEC05F0096EF3CF0AF017
:10013000040EE126300E092609C0E5FF06C0E9FFDE
:1001400007C0F3FF0850D1EC0AF0062AD8B0072AFE
:10015000D8B0082A030603500EE12E0EE56E06C045
:10016000E9FF07C0F3FF0850D1EC0AF0062AD8B027
:10017000072AD8B0082A030EE56EE80EE56E055092
:10018000E56E0450E56E4EEC05F0046EF3CF05F01D
:10019000040EE126000EE56E640EE56E0550E56E78
:1001A0000450E56EAAEC05F0096EF3CF0AF0040ED8
:1001B000E126300E092609C0E5FF06C0E9FF07C0A9
:1001C000F3FF0850D1EC0AF0062AD8B0072AD8B0BD
:1001D000082A030603500EE12E0EE56E06C0E9FF65
:1001E00007C0F3FF0850D1EC0AF0062AD8B0072A5E
:1001F000D8B0082A000EE56E640EE56E0550E56E77
:100200000450E56E4EEC05F0046EF3CF05F0040EDD
:10021000E126000EE56E0A0EE56E0550E56E04500F
:10022000E56EAAEC05F0096EF3CF0AF0040EE126A4
:10023000300E092609C0E5FF06C0E9FF07C0F3FF3D
:100240000850D1EC0AF0062AD8B0072AD8B0082AFC
:10025000030603500EE12E0EE56E06C0E9FF07C04F
:10026000F3FF0850D1EC0AF0062AD8B0072AD8B01C
:10027000082A000EE56E0A0EE56E0550E56E045084
:10028000E56E4EEC05F0046EF3CF05F0040EE126AA
:10029000300E042604C0E5FF06C0E9FF07C0F3FFE7
:1002A0000850D1EC0AF0062AD8B0072AD8B0082A9C
:1002B000032E09D02E0EE56E06C0E9FF07C0F3FF3E
:1002C0000850D1EC0AF00050040F036E000E01201C
:1002D000046E000E0220056E0250800FF36E055072
:1002E000800FF35C05E10450015C02E10350005C07
:1002F00019E200C0E9FF01C0F3FF02507AEC0AF0F6
:10030000066E300A0FE1200EE56E00C0E9FF01C065
:10031000F3FF0250D1EC0AF0002AD8B0012AD8B07D
:10032000022ADAD7E4CF0AF0E4CF09F0E4CF08F0EC
:10033000E4CF07F0E4CF06F0E4CF05F0E4CF04F01B
:10034000E4CF03F0E4CF02F0E4CF01F0E4CF00F01B
:10035000E4CFD9FF1200D9CFE5FFE1CFD9FF00C02C
:10036000E5FF01C0E5FF02C0E5FF03C0E5FF04C0F3
:10037000E5FF05C0E5FF06C0E5FF07C0E5FF020E8B
:10038000DBCF00F0030EDBCF01F0040EDBCF02F079
:10039000050EDBCF03F0640EE56E03C0E5FFC7EC8E
:1003A00008F0046EE450E450300E042604C0E5FF6B
:1003B00000C0E9FF01C0F3FF0250D1EC0AF0005089
:1003C000010F046E000E0120056E000E0220066E65
:1003D000640EE56E03C0E5FF1DEC08F0036EE4500B
:1003E000E4500A0EE56E03C0E5FFC7EC08F0076EA7
:1003F000E450E450300E072607C0E5FF04C0E9FFD3
:1004000005C0F3FF0650D1EC0AF0042AD8B0052A43
:10041000D8B0062A0A0EE56E03C0E5FF1DEC08F011
:10042000036EE450E450300E032603C0E5FF04C021
:10043000E9FF05C0F3FF0650D1EC0AF00050020FAF
:10044000036E000E0120046E000E0220056E0250A5
:10045000800FF36E0550800FF35C05E10450015CE2
:1004600002E10350005C19E200C0E9FF01C0F3FFA4
:1004700002507AEC0AF0066E300A0FE1200EE56EAB
:1004800000C0E9FF01C0F3FF0250D1EC0AF0002ADE
:10049000D8B0012AD8B0022ADAD7E4CF07F0E4CFE7
:1004A00006F0E4CF05F0E4CF04F0E4CF03F0E4CFAE
:1004B00002F0E4CF01F0E4CF00F0E4CFD9FF120066
:1004C000D9CFE5FFE1CFD9FF00C0E5FF01C0E5FFCF
:1004D00002C0E5FF03C0E5FF04C0E5FF05C0E5FF7E
:1004E00006C0E5FF07C0E5FF08C0E5FF020EDBCF51
:1004F00000F0030EDBCF01F0040EDBCF02F0050E9F
:10050000DBCF03F0060EDBCF04F0070EDBCF05F0E8
:10051000080EDBCF06F0090EDBCF07F0D0EC09F0B8
:1005200003A003D0020EC86E02D0090EC86E0CECF8
:100530000BF00050E56EB9EC0AF0E12A03A208D0F6
:100540000250036E086A0350E56EB9EC0AF0E12A26
:100550000150E56EB9EC0AF0E12A06EC0BF00080E0
:100560000050E56EB9EC0AF0E12A04C000F005C0C5
:1005700001F006C002F007C003F0020E035C16E3B0
:10058000010EE56E1FEC0AF0046EE12A04C0E5FFDF
:1005900000C0E9FF01C0F3FF0250D1EC0AF0002ACD
:1005A000D8B0012AD8B0022A0306E7D703500FE0DB
:1005B000000EE56E1FEC0AF0036EE12A03C0E5FFB2
:1005C00000C0E9FF01C0F3FF0250D1EC0AF000ECDB
:1005D0000BF0E86AE4CF08F0E4CF07F0E4CF06F0D0
:1005E000E4CF05F0E4CF04F0E4CF03F0E4CF02F071
:1005F000E4CF01F0E4CF00F0E4CFD9FF1200D9CF6F
:10060000E5FFE1CFD9FF00C0E5FF01C0E5FF02C073
:10061000E5FF03C0E5FF04C0E5FF05C0E5FF06C038
:10062000E5FF07C0E5FF08C0E5FF09C0E5FF0AC018
:10063000E5FF0BC0E5FF0CC0E5FF0DC0E5FF020EB6
:10064000DBCF00F0030EDBCF01F0040EDBCF02F0B6
:10065000050EDBCF03F0060EDBCF04F0070EDBCF79
:1006600005F0080EDBCF06F0090EDBCF07F0086AB5
:10067000096A0A6A0B6A200E0C6E0344010B0D6EA8
:10068000010E0D16005000260136023603360850C2
:10069000082609360A360B360D50D8A408800750B4
:1006A0000B5C08E106500A5C05E10550095C02E1BB
:1006B0000450085C09E30450085E0550095A0650CE
:1006C0000A5A07500B5A00800C2ED7D703C0E9FFF7
:1006D00002C0F4FF01C0F3FF0050E4CF0DF0E4CFFF
:1006E0000CF0E4CF0BF0E4CF0AF0E4CF09F0E4CF54
:1006F00008F0E4CF07F0E4CF06F0E4CF05F0E4CF54
:1007000004F0E4CF03F0E4CF02F0E4CF01F0E4CF53
:1007100000F0E4CFD9FF1200D9CFE5FFE1CFD9FF38
:1007200000C0E5FF01C0E5FF02C0E5FF03C0E5FF33
:1007300004C0E5FF05C0E5FF06C0E5FF07C0E5FF13
:10074000020EDBCF00F0030EDBCF01F0040EDBCF97
:1007500002F0050EDBCF03F0060EDBCF04F0070E30
:10076000DBCF05F0080EDBCF06F0090EDBCF07F07C
:10077000D0EC09F003A003D0020EC86E02D0090E1F
:10078000C86E0CEC0BF00050E56EB9EC0AF0E12AF3
:1007900003A208D00250006E036A0050E56EB9EC67
:1007A0000AF0E12A0150E56EB9EC0AF0E12A04C032
:1007B00000F005C001F006C002F007C003F003C05E
:1007C00004F00306045013E000C0E9FF01C0F3FF8A
:1007D00002507AEC0AF0046E002AD8B0012AD8B090
:1007E000022A0450E56EB9EC0AF0E12AE8D700ECE1
:1007F0000BF0E86AE4CF07F0E4CF06F0E4CF05F0B1
:10080000E4CF04F0E4CF03F0E4CF02F0E4CF01F052
:10081000E4CF00F0E4CFD9FF1200D9CFE5FFE1CF5C
:10082000D9FF00C0E5FF01C0E5FF02C0E5FF03C03E
:10083000E5FF04C0E5FF020EDBCF00F0030EDBCFC7
:1008400001F0040EDBCF02F0050EDBCF03F0060E45
:10085000DBCF04F0D0EC09F0090EC86E0CEC0BF005
:10086000C60EE56EB9EC0AF0E12A000EE56EB9ECB1
:100870000AF0E12AFE0EE56EB9EC0AF0E12A015019
:10088000400DF3CF01F0800E0126015000260050EC
:10089000E56EB9EC0AF0E12A02C000F003C001F0F5
:1008A00004C002F000C0E9FF01C0F3FF02507AEC7F
:1008B0000AF0036E03500BE0002AD8B0012AD8B02A
:1008C000022A0350E56EB9EC0AF0E12AEBD7FF0EDD
:1008D000E56EB9EC0AF0E12A00EC0BF0000EE56ED3
:1008E0000A0EE56E69EC09F0020EE126E4CF04F091
:1008F000E4CF03F0E4CF02F0E4CF01F0E4CF00F066
:10090000E4CFD9FF1200110E0001906F220E916FFB
:10091000330E926F440E936F620ED36E0F0E936E72
:10092000816A818EAAEC0AF034EC09F0ECEC0AF052
:10093000000EE56E130EE56E2E0EE56E000EE56EF2
:10094000000EE56E0DEC04F0050EE126020EE56EDC
:100950009DEC09F0006EF3CF01F0E12AD89001324E
:100960000032D89001320032000E036E800E026E0B
:10097000800E046E0150E56E0050E56E000EE56ECF
:100980000450E56E0350E56E0250E56E15EC00F084
:10099000060EE1260001856B000E016E800E006ED2
:1009A000800E026EE56E0150E56E0050E56E010EA0
:1009B000E56E000EE56E0DEC04F0050EE126030E6B
:1009C000E56EE80EE56E69EC09F0020EE126BED791
:1009D0001200D9CFE5FFE1CFD9FF00C0E5FF01C08C
:1009E000E5FF02C0E5FF03C0E5FF04C0E5FF05C069
:1009F000E5FF06C0E5FF07C0E5FF08C0E5FF09C049
:100A0000E5FF0AC0E5FF0BC0E5FF020EDBCF00F0FB
:100A10000050E56EA9EC07F0016EF3CF02F0E12A79
:100A2000036A046A002A002A0050E56EA9EC07F068
:100A3000006EF3CF05F0E12A066A076A05500B6ED7
:100A400000500A6E086A096A085001120950021221
:100A50000A5003120B50041204C0E9FF03C0F4FF54
:100A600002C0F3FF0150E4CF0BF0E4CF0AF0E4CF73
:100A700009F0E4CF08F0E4CF07F0E4CF06F0E4CFCC
:100A800005F0E4CF04F0E4CF03F0E4CF02F0E4CFCC
:100A900001F0E4CF00F0E4CFD9FF1200D9CFE5FF99
:100AA000E1CFD9FF00C0E5FF01C0E5FF02C0E5FFCF
:100AB00003C0E5FF04C0E5FF05C0E5FF06C0E5FF94
:100AC000020EDBCF00F0030EDBCF01F0040EDBCF14
:100AD00002F0050EDBCF03F0046A056A0344010B44
:100AE000066E06B011D00250022603360350015C98
:100AF00002E10250005C04E2D8900332023204D0DA
:100B0000052A05C004F0EAD70350015C02E1025057
:100B1000005C04E30250005E0350015AD890033297
:100B2000023204C005F004060550EEE101C0F3FFF7
:100B30000050E4CF06F0E4CF05F0E4CF04F0E4CFBA
:100B400003F0E4CF02F0E4CF01F0E4CF00F0E4CF13
:100B5000D9FF1200D9CFE5FFE1CFD9FF00C0E5FFF3
:100B600001C0E5FF02C0E5FF03C0E5FF04C0E5FFEB
:100B700005C0E5FF06C0E5FF07C0E5FF020EDBCFBD
:100B800000F0030EDBCF01F0040EDBCF02F0050E08
:100B9000DBCF03F0046A056A100E066E0144010BF8
:100BA000076E010E07160050002601360450042679
:100BB00005360750D8A404800350055C02E10250BA
:100BC000045C05E30250045E0350055A0080062EC3
:100BD000E5D701C0F3FF0050E4CF07F0E4CF06F003
:100BE000E4CF05F0E4CF04F0E4CF03F0E4CF02F06B
:100BF000E4CF01F0E4CF00F0E4CFD9FF1200D9CF69
:100C0000E5FFE1CFD9FF00C0E5FF01C0E5FF02C06D
:100C1000E5FF020EDBCF00F000380F0B016E300E47
:100C200001263A0E015C02E3070E01260150000185
:100C3000976F0F0E0014016E300E01263A0E015C04
:100C400002E3070E012601500001986F9969000E1A
:100C5000016E970E006E800E026E030EE56E02505E
:100C6000E56E0150E56E0050E56E000EE56E000E7B
:100C7000E56E000EE56EC60EE56E8CEC03F0080E18
:100C8000E126000EE56E0A0EE56E69EC09F0020E33
:100C9000E126E4CF02F0E4CF01F0E4CF00F0E4CFAE
:100CA000D9FF1200D9CFE5FFE1CFD9FF00C0E5FFA2
:100CB00001C0E5FF02C0E5FF03C0E5FF04C0E5FF9A
:100CC00005C0E5FF06C0E5FF020EDBCF00F0030E16
:100CD000DBCF01F0040EDBCF02F0050EDBCF03F01B
:100CE000060EDBCF04F00150056E0250066EE56E75
:100CF0000550E56E0050E56E6EEC07F0030EE12640
:100D0000002A002A0350016E0450026E036A046A2E
:100D10000250E56E0150E56E0050E56E6EEC07F096
:100D2000030EE126E4CF06F0E4CF05F0E4CF04F0B3
:100D3000E4CF03F0E4CF02F0E4CF01F0E4CF00F021
:100D4000E4CFD9FF1200E60EF66E150EF76E000E18
:100D5000F86E0900F550056E0900F550066E055055
:100D600002E106503BE00900F550006E0900F55025
:100D7000016E0900F550026E09000900F550E96E98
:100D80000900F550EA6E090009000900F550036EEC
:100D90000900F550046E09000900F6CF07F0F7CFFF
:100DA00008F0F8CF09F000C0F6FF01C0F7FF02C05D
:100DB000F8FF035002E1045007E00900F550EE6E21
:100DC0000306F8E20406F9D707C0F6FF08C0F7FFEC
:100DD00009C0F8FF0506C4E20606C5D71200D9CF40
:100DE000E5FFE1CFD9FF00C0E5FF01C0E5FF02C08C
:100DF000E5FF03C0E5FF04C0E5FF05C0E5FF020E07
:100E0000DBCF00F0030EDBCF01F0040EDBCF02F0EE
:100E1000050EDBCF03F0046A0350045C14E200C04B
:100E2000E9FF01C0F3FF02507AEC0AF0056E002AD8
:100E3000D8B0012AD8B0022A0550E56E68EC0AF055
:100E4000E12A042AE9D7E4CF05F0E4CF04F0E4CFA7
:100E500003F0E4CF02F0E4CF01F0E4CF00F0E4CF00
:100E6000D9FF1200D9CFE5FFE1CFD9FF00C0E5FFE0
:100E700001C0E5FF02C0E5FF020EDBCF00F000502D
:100E800000019A6F9B69000E016E9A0E006E800E33
:100E9000026E020EE56E0250E56E0150E56E0050E6
:100EA000E56E000EE56E000EE56E000EE56EC60EF8
:100EB000E56E8CEC03F0080EE126000EE56E0A0EDE
:100EC000E56E69EC09F0020EE126E4CF02F0E4CF12
:100ED00001F0E4CF00F0E4CFD9FF1200D9CFE5FF55
:100EE000E1CFD9FF00C0E5FF01C0E5FF02C0E5FF8B
:100EF000020EDBCF00F0030EDBCF01F0040EDBCFE0
:100F000002F0A69EA69CA684F29E00C0A9FF0150F6
:100F1000A86E550EA76EAA0EA76EA682A6B2FED721
:100F20000028A96E0250016E026A0150A86E550E8B
:100F3000A76EAA0EA76EA682A6B2FED7A694F28EC0
:100F4000E4CF02F0E4CF01F0E4CF00F0E4CFD9FF2A
:100F50001200D9CFE5FFE1CFD9FF00C0E5FF01C006
:100F6000E5FF02C0E5FF03C0E5FF04C0E5FF05C0E3
:100F7000E5FF020EDBCF00F0A69CA69E00C0A9FFF5
:100F8000A680A8CF01F0026A0028A96EA680A8CF8B
:100F900000F0036A0050056E046A04500112055007
:100FA000021202C0F3FF0150E4CF05F0E4CF04F0D9
:100FB000E4CF03F0E4CF02F0E4CF01F0E4CF00F09F
:100FC000E4CFD9FF1200D9CFE5FFE1CFD9FF00C0B0
:100FD000E5FF01C0E5FF02C0E5FF03C0E5FF020E2B
:100FE000DBCF00F0030EDBCF01F0040EDBCF02F00D
:100FF00000C0E9FF01C0F3FF02507AEC0AF0036E73
:10100000035010E0ACA2FED700C0E9FF01C0F3FF1F
:1010100002507AEC0AF0AD6E002AD8B0012AD8B09E
:10102000022AE6D7E4CF03F0E4CF02F0E4CF01F0E8
:10103000E4CF00F0E4CFD9FF1200D9CFE5FFE1CF34
:10104000D9FF00C0E5FF01C0E5FF02C0E5FF03C016
:10105000E5FF020EDBCF00F0030EDBCF01F0026AEA
:10106000036A01BE0CD0D89001360150005C03E247
:10107000D890013204D0032A03C002F0F2D7015005
:10108000005C02E30150005ED890013202C003F020
:1010900002060350F4E10050E4CF03F0E4CF02F085
:1010A000E4CF01F0E4CF00F0E4CFD9FF120000C09C
:1010B000E5FF01C0E5FF02C0E5FF03C0E5FFFEEC70
:1010C00008F0006EF3CF01F0F4CF02F0E9CF03F0A7
:1010D000000EE56E0F0EE56E420EE56E400EE56EFB
:1010E0000350E56E0250E56E0150E56E0050E56E6E
:1010F000FFEC02F0006EF3CF01F0F4CF02F0E9CF85
:1011000003F0080EE12601C0F3FF0050E4CF03F026
:10111000E4CF02F0E4CF01F0E4CF00F0120000C011
:10112000E5FF01C0E5FF02C0E5FF03C0E5FFFEECFF
:1011300008F0006EF3CF01F0F4CF02F0E9CF03F036
:10114000000EE56E000EE56E030EE56EE80EE56E30
:101150000350E56E0250E56E0150E56E0050E56EFD
:10116000FFEC02F0006EF3CF01F0F4CF02F0E9CF14
:1011700003F0080EE12601C0F3FF0050E4CF03F0B6
:10118000E4CF02F0E4CF01F0E4CF00F01200D9CFB9
:10119000E5FFE1CFD9FF00C0E5FF01C0E5FF02C0D8
:1011A000E5FF03C0E5FF04C0E5FF020EDBCF00F062
:1011B000030EDBCF01F0026A080E036E800E0014EE
:1011C000046ED8900036D89002360450D8A402801D
:1011D0000150025C03E30150025E0080032EEED753
:1011E0000050E4CF04F0E4CF03F0E4CF02F0E4CF0A
:1011F00001F0E4CF00F0E4CFD9FF120000C0E5FF1A
:1012000001C0E5FF02C0E5FF03C0E5FF04C0E5FF44
:1012100005C0E5FFB2CF00F0B3CF01F09CC002F0F3
:101220009DC003F0B2CF04F0B3CF05F00150055CD0
:1012300002E10050045C04E29CC002F09DC003F097
:1012400003C0E9FF02C0F4FF05C0F3FF0450E4CF80
:1012500005F0E4CF04F0E4CF03F0E4CF02F0E4CFF4
:1012600001F0E4CF00F0120000C0E5FF01C0E5FF8F
:1012700002C0E5FFFE0E0001946F010E956F9669A6
:10128000000E016E940E006E800E026E030EE56E6F
:101290000250E56E0150E56E0050E56E000EE56E01
:1012A000000EE56E000EE56EC60EE56E8CEC03F0EA
:1012B000080EE126000EE56E0A0EE56E69EC09F0F7
:1012C000020EE126E4CF02F0E4CF01F0E4CF00F01B
:1012D0001200D9CFE5FFE1CFD9FF00C0E5FF01C083
:1012E000E5FF02C0E5FF03C0E5FF020EDBCF00F023
:1012F000030EDBCF01F000C002F001C003F0FF0ECF
:101300000026D8A001060250031006E0FA0E026E75
:101310000000022EFDD7EFD7E4CF03F0E4CF02F0B8
:10132000E4CF01F0E4CF00F0E4CFD9FF1200546520
:101330006D706572617475726500D9CFE5FFE1CF9C
:10134000D9FF00C0E5FF01C0E5FF02C0E5FF03C013
:10135000E5FF020EDBCF00F00044E844FC0B016E19
:10136000030E0110C26EC2B2FED7C4CF00F0016AF4
:101370000050036E026AC3CF00F0016A00500226DB
:101380000150032203C0F3FF0250E4CF03F0E4CF87
:1013900002F0E4CF01F0E4CF00F0E4CFD9FF120077
:1013A00000C0E5FF01C0E5FF02C0E5FFFF0E006ED3
:1013B0001F0EC514016E026AC7B4022A0250011240
:1013C000015003E000060050F3E100C001F00050BE
:1013D000D8B48BEC0AF00150D880E866D890016A46
:1013E00001360150E4CF02F0E4CF01F0E4CF00F089
:1013F0001200D9CFE5FFE1CFD9FF00C0E5FF01C062
:10140000E5FF020EDBCF00F0030EDBCF01F0A69E5E
:10141000A69CA684F29E01C0A8FF00C0A9FF550E9D
:10142000A76EAA0EA76EA682A6B2FED7A694F28ECB
:10143000E4CF01F0E4CF00F0E4CFD9FF1200D9CF20
:10144000E5FFE1CFD9FF00C0E5FF01C0E5FF020ED7
:10145000DBCF00F0D0EC09F0C586D0EC09F0C9CFA5
:1014600001F0D0EC09F0005002E0C59A01D0C58A25
:10147000C5880150E4CF01F0E4CF00F0E4CFD9FFFC
:101480001200D9CFE5FFE1CFD9FF00C0E5FF020E82
:10149000DBCF00F0A69CA69E00C0A9FFA680A850A6
:1014A000E4CF00F0E4CFD9FF120000C0E5FF01C097
:1014B000E5FF1F0EC514006E016AC7B4012A015072
:1014C00000120050F6E1E4CF01F0E4CF00F012008A
:1014D000D9CFE5FFE1CFD9FF00C0E5FF020EDBCF9A
:1014E00000F0ACA2FED700C0ADFFE4CF00F0E4CF27
:1014F000D9FF1200E8AE04D0F3CFEAFFEE5012009D
:10150000E8BC08D0E9CFF6FFF3CFF7FFF86E09008B
:10151000F55012001200818AC69A9496828682B88B
:1015200003D082968286FBD794988298828894868C
:101530009488C68A1200200EAC6E900EAB6E0C0E14
:10154000AF6E000EE56E010EE56E69EC09F0020E5D
:10155000E12612003F0EC716280EC66EC56A090E98
:10156000C86E948694889E96A1968BEC0AF0819A18
:101570001200D9CFE5FFE1CFD9FF020EDBCFC9FFC3
:10158000D0EC09F0E4CFD9FF120012EEFFF022EE0A
:10159000FFF0F86AA68EA69CA3EC06F083EC04F09C
:1015A000FFD7E8AE05D0F3CFEAFFE4CFEEFF12009D
:1015B000E8AC1200120000C0E5FF006A9EBA002AE3
:1015C0000050E4CF00F01200810EB16EB36AB26A2F
:1015D00000019C6B9D6B1200010EC26E050EC16E68
:1015E000940EC06E12000100361600009E0000002E
:1015F00001000000B36AB26A00019C6B9D6B12008F
:10160000D0EC09F0C584C5B4FED71200D0EC09F0C7
:10161000C582C5B2FED71200D0EC09F0C580C5B0B6
:10162000FED7120000019C2B01E39D2B12009EAA05
:08163000FED7AE5012000000CD
:00000001FF
